:10000000400A2A08200854085208550845082008C4
:100010004408490847084908540841084C08200882
:1000200053085108550845084C084308480820085B
:1000300028084308290820083108390839083708F2
:100040002008480847083508410856085408200881
:100050002C0820084808410835084F0842082008A5
:100060002A0820082008760832082E0830082008C0
:100080003C0C0600010C2600040C02006900E90289
:10009000470A66074D0A030C4E0A040C02000400CE
:1000A0006B0028052807580A46065C0A2804650ADA
:1000B00046075C0A28056D0A81024307520A6B0055
:1000C0006100060526040400520A01022E00CD013B
:1000D0008D090E022D000400520A01026100AD00DC
:1000E0006D02AD028D090400520A2900E906820A58
:1000F000C50CCB0103067F0A0902EB0100080604C8
:1001000026050008100C8B0003078A0A09027F0EDF
:10011000AB0000080605260400082900180C890019
:100120000307980AA80C890003079A0A8A0C750A23
:10013000850C750A9D09CA01750A180C89002900E9
:10014000F00E2A00AA0309020F0EE20185088408B6
:1001500083088208810802080308040804080308C9
:0C016000020881088208830884088508D2
:0203FE00000AF3
:084000000D000C000D00020090
:02400E00E50FBC
:02FFFE000805F4
:00000001FF
